:100000008CC0B0C0AFC0AEC0ADC0B1C0ABC0AAC0A4
:10001000A9C0A8C0A7C0A6C0A5C0A4C0A3C0814550
:1000200086468B479048944997609B619E62A16386
:10003000A464A765AA66AC67AE68B069B280B481F3
:10004000B682B883BA84BB84BD84FF21000000005F
:100050000000000000000000000023456C98C9FF6C
:10006000040714233764A0FFFFFFFFFFFFFFFFFF1C
:10007000FFFFFF00000000000000000023405F7A47
:10008000B4FFFFFFFFFFFF001400081400080E1468
:100090000004080E14000305080E140004080A0EDC
:1000A0001114000305080A0E1014000305080A0EB7
:1000B0001012140008000E00080E0004080E0003C1
:1000C00005080E0004080E1100080E1100F3F404D8
:1000D000080E10121400080A0C0E0F10121400085B
:1000E0000EED14000203040500041400040E1400B5
:1000F000040810140004080F1114000305080A0E68
:100100000004080A0E00EEEDECEB140E08040004E7
:10011000080E00EBECEDEEF3F41411241FBECFE556
:10012000D2E0DEBFCDBF20E0A0E6B0E001C01D926E
:10013000AA37B207E1F7EBE7F0E085E5808781E0D9
:10014000838314821282868311828BE0818788E503
:100150008287E1E6F0E08DEF87838EEF8583712C57
:10016000B6D0C6C24DCF1BBC19BC18BC089518959B
:1001700025B7277E25BF29B7226029BF21E022BFEE
:10018000019728F020E188952150E9F7F9CF0895EB
:1001900088EE93E0EDCF369A3699FECF95B18091F7
:1001A000600089270895CF93C72D81E0870D8F7355
:1001B000782E662D90E08ED26FEF8C2F90E0CF914D
:1001C00089C2FF920F931F93CF93DF93F82E0CE712
:1001D00010E0CEE7D0E0F11005C0CE0173D2F801F7
:1001E000808304C0F8016081CE0174D221970F5F33
:1001F0001F4FC437D10579F7DF91CF911F910F9130
:10020000FF900895D0DF81E0DCCF811101C0ABCF3A
:10021000815090E0FC01E45BFF4FE491EBBDFC01F9
:10022000E05AFF4FE491E9BDFC01EC58FF4F849187
:1002300088BD08950F931F93CF93C82F8B01CC23B4
:1002400059F085E0E2DFC80193DF8DDFC80190DF60
:10025000C8018EDFC150F3CFCF911F910F91089548
:10026000EF92FF920F931F93CF93C8E0E82EF12CEB
:10027000062F10E084E1C9DFC7017ADF74DFC8010F
:1002800077DFC150B9F7CF911F910F91FF90EF9099
:1002900008951F93CF93DF938FEA87B986EC86B9D1
:1002A0001092600010E1C0E0D0E085E090E060DFF7
:1002B00072DFC80FD11D1150C1F7CE0124E0969511
:1002C00087952A95E1F7DF91CF911F9108951092BC
:1002D0007A0083EA87B986EC86B93699FECF369ADA
:1002E0003699FECF85B18095582E87E790E0EAD108
:1002F000853519F0612C86DF11C0712C872D90E0B7
:10030000E1D1682E8F3F19F080E05BDF07C0872DB9
:1003100091E0970D792E803488F3F6CF20918400F8
:10032000C0917E0010917F0080917C00882319F09D
:1003300010E0C0E02AE12F5F90E040E050E0A8E844
:10034000B0E0222379F0BD016F5F7F4FFB01319751
:10035000E491EE2319F0962F9A1BF6CF2150AD01B0
:10036000DB01EFCF092F6C2F70E0A92FB0E0E02F59
:10037000F0E0112321F09D012E1B3F0B05C09F01D2
:1003800021503109260F371F3197E40FF51FF490E4
:1003900026593F4FF901F082015049F79C0F909385
:1003A0008600CC2371F0112329F0292F30E0215051
:1003B000310902C020E030E0F901E659FF4F41E089
:1003C000408327E0290F322F3150E32FE91BF0E063
:1003D000ED5EFE4FE491A32FB0E0A659BF4FEC9322
:1003E0003913F2CFE22FF0E0E759FF4F31E050919F
:1003F0006A004081541330E0231B20938700362D80
:10040000353FE8F5452D4134B0F4809188008F3FA9
:1004100029F480917A008093880006C081E0860DDF
:10042000682E891708F0612C809188008F5F8F718A
:100430008093880024C030917A00309388004F3A2E
:10044000C0F430918100332311F0882339F081E02A
:10045000860D682E891798F0612C11C0862D6916BB
:10046000D9F3662019F08150682E09C02150622E00
:1004700006C08111F1CF80917D00882369F38FEF51
:100480008DBD80E68CBD8FE384BB8BE187BB8CEE9A
:1004900088BB81E083BF91EA9ABD80BF85B7806247
:1004A00085BF78948CE287B986EC86B93699FECF01
:1004B0008FEF80936000C62DC53F10F0612C3CC0CB
:1004C00080918800803138F4E62DF0E0E659FF4F46
:1004D000C081DC2F31C05CDE80917A00809388007F
:1004E000CCE7D0E000E010E0FF24F39481E0800F3F
:1004F0000F5F1F4F98819F3F29F421960830110507
:10050000A9F7E2CF6DE570E095DEF801EF59FF4FF6
:10051000608088818F25888375DE6FE070E080E2DF
:1005200089DE88818F258883612C6CDE31DE8091A5
:100530007C00882311F3C8CF36DE10E0F12C8CE26A
:10054000D82E96ECC92EEE24EA94CE3E19F463E43C
:1005500081E204C0CD3E21F468E284E181DE76C010
:10056000CC3E11F469E203C0CB3E19F462E581E0B0
:10057000F5CFC33F81F404E084E147DE85E090E0FD
:10058000F7DD88E042DE81E490E0F2DD0150A1F782
:1005900080ED92E05AC0C43F51F584E690E0E8DD7A
:1005A000FADD90E0292F30E0F901E25EFF4FE4919F
:1005B000E81710F49E5FF6CFF901E15EFF4F04915A
:1005C0006DE770E0802F82958695877033DE8EEE22
:1005D00092E0CEDD65E070E081E02CDE85E694E01F
:1005E000C7DD6DE770E0802F8F7124DE0DC0CE3F38
:1005F00071F400E00093840005DE6AEF70E081E0B2
:1006000019DE0F5F0A31B1F7C3DDC2DD1FC0CD3F78
:1006100069F58FEF80938500F5DD85E0F6DDB8DDC7
:10062000B7DD84E1F2DD35DE80938500EBDDB0DD02
:10063000AFDDF9CF3699FECFE0926000F394909150
:1006400085008917C8F484EF91E092DD80917A00EB
:1006500080938800A0DD803998F51F5F183008F47A
:1006600074CFD53190F010E0DAE0CAE08D2FCDDD07
:1006700010DED7B8C6B8DECFDB3028F3F4E1FF15C3
:1006800010F7E0927A00DAE0DECFD23030F08D2F32
:1006900086958695D695D80F12C065DD85B7877E7D
:1006A000806185BFF89485B7846885BF8B7F85BFDF
:1006B00085B7806285BF889585B78F7D85BFCD2F33
:1006C00010E043CFE199FECF9FBB8EBBE09A992704
:1006D0008DB30895262FE199FECF1CBA9FBB8EBB28
:1006E0002DBB0FB6F894E29AE19A0FBE01960895D9
:0406F000F894FFCFAC
:00000001FF
